:0A00000075817F7401F58F02000E78
:10000B0002096375F15490000074F2F0A37407F0C9
:10001B0090000274F2F0A37407F090000474F2F0F5
:10002B00A37407F0120186C209C23FC206C207C2FF
:10003B00081201721210BB12123512146D120172DA
:10004B00120172120172120172C2B6C2B5C2B7129C
:10005B00119B1211CC1211FDD2B6D2B5D2B712012F
:10006B0072120172120172120172C215C216C217FC
:10007B007590FB75A0FFD2B4C20FC212C210C2138F
:10008B00C211C214C200C202C204C201C203C20521
:10009B00C206C207C208C209C20AC20BD227D228A3
:1000AB00D229C22DC22EC22FC23FC240C241D22181
:1000BB00D222D223C23CC23DC23ED218D219D21A8E
:1000CB00120172120931D22AD22BD22C7565C87546
:1000DB0067C87569C874328575F0A4F55CF55DF574
:1000EB005E2412F55FF560F5617400900006F090E8
:1000FB000007F0900008F07480F562F563F564C2B8
:10010B0043C244C245754200754300753A00753BC6
:10011B0000120500120538120570854244854345CF
:10012B001205B012017212017212017212127012C8
:10013B0003841203961203A8120500120538120548
:10014B007012051C1205541202BE1202E512030CAA
:10015B001205B01205DB120606020137783279FF61
:10016B000000D9FCD8F822786479FF0000D9FCD8BC
:10017B00F822781E7996D9FED8FA22C2B6D2B5D219
:10018B00B7120172120172C2B6C2B5D2B7120172A6
:10019B00120172C2B6C2B5C2B7120172120172124B
:1001AB000172120172C2B6C2B5D2B712017212013C
:1001BB0072C2B6D2B5D2B7120172120172D2B6D2D6
:1001CB00B5D2B712017212017212017212017222B0
:1001DB00E627F5290809E637F52A782922C3E69799
:1001EB00F5290809E697F52A7829228629872B080D
:1001FB0009862A872C12027B782E22862E08862FC0
:10020B00088630088631872B09872C12021E782925
:10021B0079302275320075331012026012023112DE
:10022B000254D533F422C3E530952BE531952CE5FB
:10023B00329400500122E530952BF530E531952CA9
:10024B00F531E5329400F53222B3E52933F529E592
:10025B002A33F52A22C3E52E33F52EE52F33F52F5E
:10026B00E53033F530E53133F531E53233F5322214
:10027B00E529852BF0A4F52E85F02FE52A852CF0AA
:08028B00A4F53085F031E52AED
:10029300852BF0A4252FF52FE53035F0F530E5312A
:1002A3003400F531E529852CF0A4252FF52FE53011
:1002B30035F0F530E5313400F53122120ADD200C3A
:1002C3000122C20C30000C12063112066A12068D8E
:1002D300D2122212069D1206AF1206D8D20F1204B2
:1002E3002022120B32200D0122C20D30020C120605
:1002F300F012072912074CD2132212075C12076E61
:10030300120797D21012046D22120B87200E0122BE
:10031300C20E30040C1207AF1207E812080BD214F6
:100323002212081B12082D120856D2111204BA22E7
:1003330030410122208110200110B200D20120009F
:1003430005C218D2242222C20122223041012220D6
:100353008010200310B202D203200205C219D22555
:100363002222C203222230410122209010200510B4
:10037300B204D205200405C21AD2262222C20522C3
:10038300223000012220A708203C07D23CD21222AF
:10039300C23C223002012220A708203D07D23DD2D1
:1003A3001322C23D223004012220A708203E07D297
:1003B3003ED21422C23E22308412200912202D077D
:1003C300D218D209C24322D209C22D22C209222243
:1003D300308512200A12202E07D219D20AC24422D3
:1003E300D20AC22E22C20A2222308212200B1220EB
:1003F3002F07D21AD20BC24522D20BC22F22C20B15
:100403002222208614200614B221D206D22DC21B2A
:10041300C21CC230C231D24322C206222220181784
:10042300C215C2B6202108120BFD88448945221249
:100433000C728844894522855C5F74328575F0A40B
:10044300F55CC215D2B6A842A94388448945222047
:100453008714200714B222D207D22EC21DC21EC295
:0804630032C233D24422C20769
:10046B002222201917C216C2B5202208120D23888A
:10047B0046894722120D988846894722855D60740C
:10048B00328575F0A4F55DC216D2B5A83CA93D889E
:10049B0046894722208314200814B223D208D22F76
:1004AB00C21FC220C234C235D24522C2082222202A
:1004BB001A17C217C2B7202308120E498848894958
:1004CB0022120EBE8848894922855E617432857579
:1004DB00F0A4F55EC217D2B7A83EA93F8848894958
:1004EB00227A0FC294D2A2A2A133C933C9C2A2DA13
:1004FB00F2F8D29422D2947A0574E0C2A2C2943359
:10050B0092A0D2A2DAF51204EC8840894153410F34
:10051B0022D2947A0574E8C2A2C2943392A0D2A2DA
:10052B00DAF51204EC883C893D533D0F22D2947AC4
:10053B000574F0C2A2C2943392A0D2A2DAF51204CF
:10054B00EC883A893B533B0F22D2947A0574F8C25C
:10055B00A2C2943392A0D2A2DAF51204EC883E899F
:10056B003F533F0F22853A34853B357834854038ED
:10057B0085413979381201DB86F008E6120F9FF5B9
:10058B004385F042228540348541357834853A38AD
:10059B00853B3979381201E886F008E6120FACF585
:1005AB004385F04222A844A945D295D2A4E94470D0
:1005BB007A08C2A3C296339297D2A3DAF57A08E8E7
:1005CB00C2A3C296339297D2A3DAF5C295D29622E2
:1005DB00A846A947D295D2A4E944F07A08C2A3C28F
:1005EB0096339297D2A3DAF57A08E8C2A3C2963370
:1005FB009297D2A3DAF5C295D29622A848A949D2EE
:10060B0095D296E944707A08C2A3C2A4339297D2CA
:10061B00A3DAF57A08E8C2A3C2A4339297D2A3DA7D
:10062B00F5C295D2A422200F0122D215C20FC21BF4
:10063B00C21CC230C23174328575F0A4F55C9000D7
:10064B0006F02412F55FC2437480F562120BDC9046
:10065B000000858250858351754AFF754B142285A6
:10066B005082855183A9431208D4A3A8421208E4EF
:10067B00A38582508583518550568551578844896F
:10068B004522D54A0C754AFFD54B06C200D22AC269
:10069B00182220120122C2129000008582508583FD
:1006AB0051D22A22302A1D85508285518312090F7F
:0D06BB00A3120920A3858250858351887108
:1006C8008972886B896C22A86BA96C8871897222DF
:1006D800E556B58212E557B5830D302408D21212BB
:1006E800069DD22A22C22A2220100122D216C21026
:1006F800C21DC21EC232C23374328575F0A4F55DC4
:10070800900007F02412F560C2447480F563120B60
:10071800E790283C858252858353754CFF754D14AC
:1007280022855282855383A93D1208D4A3A83C127E
:1007380008E4A38582528583538552588553598886
:1007480046894722D54C0C754CFFD54D06C202D2BE
:100758002BC2192220130122C21390283C858252F1
:10076800858353D22B22302B1D85528285538312C9
:10077800090FA3120920A3858252858353887189A2
:1007880072886D896E22A86DA96E8871897222E5BA
:1007980058B58212E559B5830D302508D2131207D2
:1007A8005CD22B22C22B2220110122D217C211C2E5
:1007B8001FC220C234C23574328575F0A4F55E902C
:1007C8000008F02412F561C2457480F564120BF23A
:1007D800905078858254858355754EFF754F142245
:1007E800855482855583A93F1208D4A3A83E1208D0
:1007F800E4A385825485835585545A85555B88487A
:10080800894922D54E0C754EFFD54F06C204D22C0D
:10081800C21A2220140122C214905078858254856D
:100828008355D22C22302C1D85548285558312097C
:100838000FA3120920A38582548583558871897274
:10084800886F897022A86FA9708871897222E55A09
:10085800B58212E55BB5830D302608D21412081B49
:05086800D22C22C22C7D
:10086D00220000D2B3000000000000C2B32200003D
:10087D00D2B3000000000000A2B4C2B3227E027AFF
:10088D0008EE3392B1FE12086EDAF622AE837A08C4
:10089D00EE3392B1FE12086EDAF6AE827A08EE33BE
:1008AD0092B1FE12086EDAF622E9FE7A08EE339264
:1008BD00B1FE12086EDAF622E8FE7A08EE3392B136
:1008CD00FE12086EDAF622D2B2C2B012088A1208EF
:1008DD00991208B6D2B022D2B2C2B012088A12084A
:1008ED00991208C5D2B0227E037A08EE3392B1FE7A
:1008FD0012086EDAF6227A0812087BEE33FEDAF869
:10090D00F422D2B2C2B01208F4120899120903F9F6
:10091D00D2B022D2B2C2B01208F412089912090351
:10092D00F8D2B022758790758922759850758C38DC
:10093D00758A38C0D043D008781479647A197B321F
:10094D007C197D02D0D0756500756700756900D280
:10095D008CD2A9D2AF22C0E0C0D043D008DD557DE6
:10096D0002D83F78191209D6120A25120A741203F9
:10097D00BA1203D31203EC12033312034E1203699E
:10098D000565E565120F6FF5650567E567120F6F74
:10099D00F5670569E569120F6FF569DC057C1912BC
:1009AD0009C6D904A95CD20CDA04AA5DD20DDB0408
:1009BD00AB5ED20ED0D0D0E032301502B2B63016CA
:1009CD0002B2B5301702B2B72230000122208404E2
:1009DD001204052220862220062D900006E0F55CEB
:1009ED00D212D206D227756500756600D224C218C0
:1009FD00C21BC21CC230C23122C206302709C22717
:100A0D00856566120A152222E566B42803020A22BC
:100A1D005003C22422D22422300201222085041246
:100A2D0004522220872220072D900007E0F55DD289
:100A3D0013D207D228756700756800D225C219C276
:100A4D001DC21EC232C23322C207302809C22885F8
:100A5D006768120A642222E568B42803020A7150FD
:100A6D0003C22522D2252230040122208204120441
:100A7D009F2220832220082D900008E0F55ED214DD
:100A8D00D208D229756900756A00D226C21AC21F12
:100A9D00C220C234C23522C208302909C229856953
:100AAD006A120AB32222E56AB42803020AC050036F
:100ABD00C22622D22622E582C4540FF9E583C469E9
:100ACD002275F0058475F002A48575F0A424122218
:100ADD00300001223018012220210122853A828521
:100AED003B83120AC3F4120ACE301B0BF55FF55C83
:100AFD00900006F0C21C22201C10D21CB55F03D240
:100B0D001B225003C23922D2392220390CB55F0382
:100B1D00D21B22500122D21B22B55F03D21B2250C1
:100B2D0003D21B2222300201223019012220220180
:100B3D0022853C82853D83120AC3F4120ACE301DF4
:100B4D000BF560F55D900007F0C21E22201E10D23D
:100B5D001EB56003D21D225003C23A22D23A222082
:0D0B6D003A0CB56003D21D22500122D21DAA
:100B7A0022B56003D21D225003D21D222230040165
:100B8A0022301A012220230122853E82853F8312C8
:100B9A000AC3F4120ACE301F0BF561F55E90000805
:100BAA00F0C22022202010D220B56103D21F225089
:100BBA0003C23B22D23B22203B0CB56103D21F2247
:100BCA00500122D21F22B56103D21F225003D21F25
:100BDA00222290000074F2F0A37407F0229000021F
:100BEA0074F2F0A37407F02290000474F2F0A37474
:100BFA0007F02230210122853A82853B83120AC3FB
:100C0A0030301CF56275F080846006120CE7020C25
:100C1A001E120CAB900000E53AF0A3E53BF022204F
:100C2A003119D231B56206D230120C76225006C280
:100C3A0036120C7622D236120C7622203615B5627E
:100C4A0006D230120C76225004120C7622D23012BE
:100C5A000C7622B56206D230120C76225006D230B9
:100C6A00120C7622120C762220430122900000E018
:100C7A00F582900001E0F583120AC375F080846062
:100C8A0010900000E0F534900001E0F535120CED0B
:100C9A0022900000E0F538900001E0F539120CB11D
:100CAA0022853A38853B39793875340075350875A7
:100CBA00360075370078341201E8863808863979A3
:100CCA003885713485723575360075370078341277
:100CDA0001E886F008E6120FACF9A8F022853A344A
:100CEA00853B3575360075370078347538007539A7
:100CFA000879381201E88634088635753600753762
:100D0A0000783485713885723979381201DB86F0BA
:100D1A0008E6120F9FF9A8F02230220122853C82B0
:100D2A00853D83120AC330321CF56375F0808460F6
:100D3A0006120E0D020D44120DD1900002E53CF090
:100D4A00A3E53DF022203319D233B56306D232121D
:100D5A000D9C225006C237120D9C22D237120D9CCE
:100D6A0022203715B56306D232120D9C2250041286
:100D7A000D9C22D232120D9C22B56306D232120D7C
:100D8A009C225006D232120D9C22120D9C22204423
:100D9A000122900002E0F582900003E0F583120A36
:100DAA00C375F080846010900002E0F5349000036F
:100DBA00E0F535120E1322900002E0F53890000398
:100DCA00E0F539120DD722853C38853D39793875D9
:100DDA00340075350875360075370078341201E825
:090DEA00863808863979388571D4
:100DF3003485723575360075370078341201E8860C
:100E0300F008E6120FACF9A8F022853C34853D3595
:100E130075360075370078347538007539087938B8
:100E23001201E88634088635753600753700783444
:100E330085713885723979381201DB86F008E6123C
:100E43000F9FF9A8F02230230122853E82853F833C
:100E5300120AC330341CF56475F080846006120FE7
:100E630033020E6A120EF7900004E53EF0A3E53F4D
:100E7300F022203519D235B56406D234120EC222BF
:100E83005006C238120EC222D238120EC2222038A5
:100E930015B56406D234120EC2225004120EC222B9
:100EA300D234120EC222B56406D234120EC22250BC
:100EB30006D234120EC222120EC222204501229003
:100EC3000004E0F582900005E0F583120AC375F093
:100ED30080846010900004E0F534900005E0F5355F
:100EE300120F3922900004E0F538900005E0F5393F
:100EF300120EFD22853E38853F39793875340075E9
:100F0300350875360075370078341201E8863808DD
:100F130086397938857134857235753600753700B1
:100F230078341201E886F008E6120FACF9A8F02233
:100F3300853E34853F35753600753700783475380E
:100F43000075390879381201E88634088635753614
:100F53000075370078348571388572397938120114
:100F6300DB86F008E6120F9FF9A8F022B4C801222D
:100F730050012274C822B43201225003743222B4C5
:100F8300C8012250012274C822B4100122500374F4
:100F93001022B4C8012250012274C822B40F0122C6
:100FA300500122740F75F0FF22B40F012250012269
:100FB300740075F0002212108D74A0F912105A12E9
:100FC30010A9E573F912105A1210A9E574F9121059
:100FD3005A1210A912108D74A1F912105A1210A9E5
:100FE30012104D1210A912107F2212108D74A0F945
:100FF30012105A1210A3E573F912105A1210A3E536
:1010030074F912105A1210A312108D74A1F9121050
:101013005A1210A312104D1210A912107F22E9FACE
:1010230012108D74A0F912105A1210A9E573F91257
:10103300105A1210A9E574F912105A1210A9EAF9FC
:1010430012105A1210A912107F22D291780812108E
:10105300AFE933F9D8F8227808E9339291F91210FD
:10106300AFD8F6227B80DB02800E12108D74A0F9BC
:1010730012105A1210A940EE12107F22C29100D210
:1010830092000000000000D29122D29100D292007F
:101093000000000000C291000000000000C2922284
:1010A300C2911210AF22D2911210AF220000D2923D
:1010B300000000A291C2922220A52C203FFAC2B6C2
:1010C300C2B5C2B71210ED12112712116112122EFE
:1010D300120172120172120172120172D2B6D2B5EA
:1010E300D2B7D23F0210BBC23F22900000754A190B
:1010F300754B018583738582747900121021121058
:1011030067A3858373858274790012102112106797
:10111300A3858256858357D54AD9754A19D54BD3AA
:101123001213082290283C754C19754D0185837361
:101133008582747900121021121067A38583738549
:1011430082747900121021121067A3858258858357
:1011530059D54CD9754C19D54DD31213292290501A
:0E11630078754E19754F0185837385827479F6
:1011710000121021121067A3858373858274790090
:10118100121021121067A385825A85835BD54ED92F
:10119100754E19D54FD312134A2212136B900000CA
:1011A100858373858274120FEDE9F91208D4A38542
:1011B1008373858274120FEDE9F81208E4A3E556F2
:1011C100B582DDE557B583D8D22A2212138690283D
:1011D1003C858373858274120FEDE9F91208D4A35B
:1011E100858373858274120FEDE9F81208E4A3E593
:1011F10058B582DDE559B583D8D22B221213A190BF
:101201005078858373858274120FEDE9F91208D441
:10121100A3858373858274120FEDE9F81208E4A3A4
:10122100E55AB582DDE55BB583D8D22C227575010F
:1012310012145B2212123C1212562220861420062E
:10124100FAC2B6D2B5D2B775750112145BD20602D5
:10125100123CC206222087142007FAD2B6C2B5D2A8
:10126100B775750212145BD207021256C20722200B
:10127100A5242018012220190122201A0122300060
:1012810001223002012230040122D241203F1DD22D
:101291003FD240C24222C23F304014C2401212EC3F
:1012A1003081FD3080FA3090F7C241221212B12212
:1012B1003042012220810FC2B6120172D2151213DF
:1012C100BCD2B6D2422220800FC2B5120172D21610
:1012D1001213F1D2B5D2422220900FC2B71201727D
:1012E100D217121426D2B7D242222230420122D280
:1012F10015D216D2171213BC1213F1121426D2B63C
:10130100D2B5D2B7D24222907850A956858373853F
:101311008274121021121067A3A9578583738582E5
:101321007412102112106722907852A95885837384
:10133100858274121021121067A3A95985837385C0
:10134100827412102112106722907854A95A858351
:1013510073858274121021121067A3A95B858373B0
:101361008582741210211210672290785085837340
:10137100858274120FED8956A38583738582741259
:101381000FED895722907852858373858274120FED
:10139100ED8958A3858373858274120FED895922D3
:1013A100907854858373858274120FED895AA385D1
:1013B1008373858274120FED895B221213089000EA
:1013C1000012090F858373858274E9F912102112C5
:1013D1001067A3120920858373858274E8F91210BE
:1013E10021121067A3E556B582D7E557B583D222FE
:1013F10012132990283C12090F858373858274E9A1
:10140100F9121021121067A31209208583738582B6
:1014110074E8F9121021121067A3E558B582D7E5D7
:1014210059B583D22212134A90507812090F85833D
:1014310073858274E9F9121021121067A312092031
:10144100858373858274E8F9121021121067A3E570
:101451005AB582D7E55BB583D222907FFFA9758506
:10146100837385827412102112106722907FFF8589
:101471008373858274120FED897512147F22E575CD
:10148100C394016019D2B6C2B5D2B712017212016A
:1014910072120172120172D2B6D2B5D2B722C2B69D
:1014A100D2B5D2B712017212017212017212017217
:1014B100D2B6D2B5D2B722464C414D45204B4E4F04
:1014C100425245434F524445522D43332D4D4F44D3
:1014D100554C45204555524F205241434B205645CE
:0E14E1005253494F4E202D20323031312056CB
:1014EF00455253494F4E20312E3032202863296206
:0814FF007920616D70657265D2
:00000001FF
